:100000000CC026C025C024C023C022C021C020C0EF
:100010001FC0B0C41DC06DC41BC011241FBECFE5DE
:10002000D2E0DEBFCDBF10E0A0E6B0E0E0E8FEE049
:1000300003C0C89531960D92A036B107D1F710E0F4
:10004000A0E6B0E001C01D92A63FB107E1F747C0AE
:10005000D7CFCF93DF93CDB7DEB725970FB6F89400
:10006000DEBF0FBECDBF89839A836B838DD3F92FFB
:10007000E82F8B81282F332784819581821793075E
:10008000A8F381E08D838D81843008F01FC081E06A
:100090008C838C81853008F015C08D819927282F9D
:1000A000392F220F331F220F331F8C819927281BD2
:1000B000390B89819A81820F931F95D38C818F5F31
:1000C0008C83E7CF8D818F5F8D83DDCF25960FB633
:1000D000F894DEBF0FBECDBFDF91CF910895CBE383
:1000E000D2E0DEBFCDBF19821E861F86188A198A0C
:1000F0001A8A1B8A1C8A1D8A1E8A1F8A188E198ECC
:100100001A8E1B8E1C8E1D8E1E8E1F8E18A219A27B
:100110001AA297D260E072EC81E090E0E0D2B5D014
:1001200027D194D38981282F33272BA33CA38BA1DC
:100130009CA181309105B9F02BA13CA12230310561
:100140002CF48BA19CA1009739F09BC02BA13CA162
:1001500022303105E9F195C084D3882309F091C09C
:1001600081E089838EC08C2F9D2F02966CE071DF19
:100170008C2F9D2F02962C2F3D2F225F3F4F44E066
:1001800050E0682F792F932F822F17D68C2F9D2F19
:10019000029604962C2F3D2F2E5E3F4F44E050E0F8
:1001A000682F792F932F822F08D68C2F9D2F0296A0
:1001B00008962C2F3D2F2A5E3F4F44E050E0682FD9
:1001C000792F932F822FF9D541D382E0898359C0AB
:1001D000E4D08FEF8AA31E8E1F8E18A219A22A893F
:1001E0003B894C895D898E899F89A88DB98D281B93
:1001F000390B4A0B5B0B8A8D9B8DAC8DBD8D8217A5
:100200009307A407B50708F03BC02E893F89488DA6
:10021000598D6E8D7F8D88A199A1DAD5262F372F24
:10022000482F592F8E859F85A889B989820F931FE2
:10023000A41FB51F8A8F9B8FAC8FBD8F8E8D9F8D16
:10024000A8A1B9A10196A11DB11D8E8F9F8FA8A352
:10025000B9A36A8D7B8D8C8D9D8D52D18AA1882307
:1002600031F468E979E080E090E0C6D106C060EF43
:100270007FE580E090E0C0D11AA214D097D2AFCF32
:10028000198284E290E09CD14DCFCF93DF93CDB71C
:10029000DEB780EB8093370080E580932D00DF91FF
:1002A000CF910895CF93DF93CDB7DEB721970FB6E7
:1002B000F894DEBF0FBECDBFF894809138008860FF
:1002C0008093380081E063D180913800877F8093EC
:1002D00038008EE090E074D18FEF80932F008091F2
:1002E0002F00898378948981992721960FB6F894F5
:1002F000DEBF0FBECDBFDF91CF910895CF93DF93C7
:10030000CDB7DEB721970FB6F894DEBF0FBECDBFD5
:10031000F8948091380088608093380081E037D16C
:1003200080913800877F8093380081E030D18091C0
:10033000380088608093380081E029D180913800AE
:10034000877F809338008EE090E03AD18FEF8093E2
:100350002F0080912F008983789489819927219695
:100360000FB6F894DEBF0FBECDBFDF91CF910895D9
:10037000CF93DF93CDB7DEB780EB80933A00109236
:100380003B008FEF809334001092350081E090E0C5
:1003900017D103D0DF91CF910895CF93DF93CDB7DD
:1003A000DEB7F89480913B00806880933B0081E049
:1003B00090E006D19FE780913B00892380933B002A
:1003C00081E090E0FDD07894DF91CF910895CF93B4
:1003D000DF93CDB7DEB727970FB6F894DEBF0FBE19
:1003E000CDBF89839A83F89483E080933500809110
:1003F0003B00806180933B00C2D080913B008F7EA8
:1004000080933B0081E090E0DBD080913B008062F4
:1004100080933B00B4D080913B008F7D80933B0064
:1004200081E090E0CDD01B821C828B819C81853045
:1004300091050CF04BC029813A818B819C81F32F6F
:10044000E22FE80FF91F80818F831D821E828D812C
:100450009E81883091050CF032C08F81282F332780
:1004600081E090E00D8002C0880F991F0A94E2F7A6
:10047000532F422F4823592327E030E08D819E815E
:10048000281B390B932F822F02C0440F551F8A95CA
:10049000E2F7952F842F8093350071D080913B0037
:1004A000806180933B006BD080913B008F7E809376
:1004B0003B008D819E8101968D839E83C8CF5FD046
:1004C0008B819C8101968B839C83AFCF10923500EA
:1004D00080913B00806280933B0051D080913B0033
:1004E0008F7D80933B0081E090E06AD078942796DE
:1004F0000FB6F894DEBF0FBECDBFDF91CF91089548
:10050000CF93DF93CDB7DEB72C970FB6F894DEBF4D
:100510000FBECDBF69837A838B839C8381E08987FB
:100520008C2F9D2F01968B879C871A868A85843015
:1005300008F018C08A85282F33278C2F9D2F01960D
:10054000820F931FB92FA82F1496EB85FC8580810D
:100550008C938B859C8501968B879C878A858F5F82
:100560008A87E4CF8C2F9D2F059631DF2C960FB60E
:10057000F894DEBF0FBECDBFDF91CF910895CF932A
:10058000DF93CDB7DEB70000DF91CF910895CF9311
:10059000DF93CDB7DEB721970FB6F894DEBF0FBE5D
:1005A000CDBF89838981811511F08A95F1F7219654
:1005B0000FB6F894DEBF0FBECDBFDF91CF91089587
:1005C000CF93DF93CDB7DEB722970FB6F894DEBF97
:1005D0000FBECDBF89839A8389819A818115910548
:1005E00011F00197F1F722960FB6F894DEBF0FBE17
:1005F000CDBFDF91CF910895CF93DF93CDB7DEB715
:1006000024970FB6F894DEBF0FBECDBF69837A83FF
:100610008B839C8389819A81AB81BC8181159105F3
:10062000A105B10529F081509040A040B040D9F714
:1006300024960FB6F894DEBF0FBECDBFDF91CF91E9
:100640000895CF93DF93CDB7DEB719D01092E100B4
:100650001092E00088ED80932A0060E875E280E067
:1006600090E03DD08FEF8093E2001092EB0010926B
:10067000F5001092F4007894DF91CF910895CF9314
:10068000DF93CDB7DEB740E450E060E670E083EE84
:1006900090E0BED140E450E060EA70E08CEE90E083
:1006A000B7D1DF91CF910895CF93DF93CDB7DEB768
:1006B00022970FB6F894DEBF0FBECDBF89839A8311
:1006C00089819A819093E1008093E00022960FB691
:1006D000F894DEBF0FBECDBFDF91CF910895EF92AA
:1006E000FF920F931F93CF93DF93CDB7DEB724977D
:1006F0000FB6F894DEBF0FBECDBF69837A838B83BC
:100700009C8389819A81AB81BC81689412F8880F9F
:10071000991FAA1FBB1F1694D1F70F2EF0E0EF2EE2
:10072000F0E8FF2EF0E70F2FF0E01F2FF02DE80E7E
:10073000F91E0A1F1B1F89819A81AB81BC81282F5A
:10074000392F4A2F5B2F689413F8220F331F441F51
:10075000551F1694D1F7912F802F7F2D6E2D69D3C1
:10076000B52FA42F932F822F815080932900249698
:100770000FB6F894DEBF0FBECDBFDF91CF911F91B2
:100780000F91FF90EF900895CF93DF93CDB7DEB731
:1007900083EE90E0DF91CF910895CF93DF93CDB7B3
:1007A000DEB78CEE90E0DF91CF910895CF93DF9389
:1007B000CDB7DEB721970FB6F894DEBF0FBECDBF21
:1007C00089838091E2008823E1F3898180932C0062
:1007D0001092E20021960FB6F894DEBF0FBECDBF97
:1007E000DF91CF910895CF93DF93CDB7DEB72497F4
:1007F0000FB6F894DEBF0FBECDBF89839A83809178
:10080000E5009091E6000097A1F08091E7009091BB
:10081000E800009759F083EE90E027D1E981FA8152
:1008200080838FEF90E08B839C8305C01B821C82AA
:1008300002C01B821C828B819C8124960FB6F89487
:10084000DEBF0FBECDBFDF91CF910895CF93DF9371
:10085000CDB7DEB71092E8001092E700DF91CF919C
:100860000895CF93DF93CDB7DEB722970FB6F894F4
:10087000DEBF0FBECDBF8091E7009091E8000097EA
:1008800029F48FEF90E089839A8302C019821A823B
:1008900089819A8122960FB6F894DEBF0FBECDBF34
:1008A000DF91CF910895CF93DF93CDB7DEB7219736
:1008B0000FB6F894DEBF0FBECDBF898369818CEE81
:1008C00090E0DCD121960FB6F894DEBF0FBECDBF0D
:1008D000DF91CF910895CF93DF93CDB7DEB78FEF40
:1008E0008093EB008CEE90E0C0D060DFDF91CF9181
:1008F00008951F920F920FB60F9211242F933F93DA
:100900004F935F936F937F938F939F93AF93BF9317
:10091000EF93FF93CF93DF93CDB7DEB78091EB00DA
:10092000882391F08091F0009091F100009731F0D0
:100930008CEE90E09AD080932C0009C01092EB00CE
:100940008FEF8093E20003C08FEF8093E200DF918E
:10095000CF91FF91EF91BF91AF919F918F917F9137
:100960006F915F914F913F912F910F900FBE0F901C
:100970001F9018951F920F920FB60F9211242F936C
:100980003F934F935F936F937F938F939F93AF9317
:10099000BF93EF93FF93CF93DF93CDB7DEB721974C
:1009A000DEBFCDBF80912C0089838091E0009091C3
:1009B000E100009739F0E091E000F091E1008981D9
:1009C00009950FC0698183EE90E058D1882349F4DE
:1009D0008091F4009091F50001969093F50080933A
:1009E000F4002196F894DEBFCDBFDF91CF91FF9147
:1009F000EF91BF91AF919F918F917F916F915F9197
:100A00004F913F912F910F900FBE0F901F9018950F
:100A1000CF93DF93CDB7DEB726970FB6F894DEBF3E
:100A20000FBECDBF89839A836B837C834D835E83A6
:100A3000E981FA818B819C8180839183E981FA81AC
:100A40008D819E8182839383E981FA811682178248
:100A5000E981FA811482158226960FB6F894DEBFDA
:100A60000FBECDBFDF91CF9108950F931F93CF930A
:100A7000DF93CDB7DEB723970FB6F894DEBF0FBE76
:100A8000CDBF89839A831B82E981FA818481958114
:100A9000009709F446C0E981FA81A981BA812081D1
:100AA0003181FB2FEA2F86819781F32FE22FE80F08
:100AB000F91F80818B83A981BA81E981FA818681BE
:100AC00097810196FB2FEA2F86839783E981FA812C
:100AD000A981BA8126813781FB2FEA2F82819381F8
:100AE0002817390798F009811A81E981FA81A981CB
:100AF000BA8186819781FB2FEA2F22813381732F60
:100B0000622F81D1F12FE02F86839783A981BA814B
:100B1000E981FA81848195810197FB2FEA2F8483F3
:100B200095838B81992723960FB6F894DEBF0FBE6D
:100B3000CDBFDF91CF911F910F9108950F931F9318
:100B4000CF93DF93CDB7DEB724970FB6F894DEBF0F
:100B50000FBECDBF89839A836B837C83E981FA8141
:100B60002B813C81848195812817390708F03FC08B
:100B7000A981BA81E981FA81268137818B819C81A3
:100B8000820F931FFB2FEA2F86839783E981FA81D7
:100B9000A981BA8126813781FB2FEA2F8281938137
:100BA0002817390798F009811A81E981FA81A9810A
:100BB000BA8186819781FB2FEA2F22813381732F9F
:100BC000622F21D1F12FE02F86839783A981BA81EB
:100BD000E981FA81248135818B819C81281B390B25
:100BE000932F822FFB2FEA2F8483958304C0E98102
:100BF000FA811482158224960FB6F894DEBF0FBED8
:100C0000CDBFDF91CF911F910F9108950F931F9347
:100C1000CF93DF93CDB7DEB724970FB6F894DEBF3E
:100C20000FBECDBF89839A836B837C8309811A8130
:100C3000E981FA81268137818B819C81820F931F04
:100C4000E981FA8122813381732F622FDCD0282F32
:100C5000392FF12FE02F80819181F32FE22FE80FC0
:100C6000F91F8081992724960FB6F894DEBF0FBE36
:100C7000CDBFDF91CF911F910F9108950F931F93D7
:100C8000CF93DF93CDB7DEB725970FB6F894DEBFCD
:100C90000FBECDBF89839A836B83E981FA81A981D5
:100CA000BA8124813581FB2FEA2F82819381281715
:100CB000390788F509811A81E981FA81A981BA8108
:100CC00026813781FB2FEA2F84819581820F931F24
:100CD000E981FA8122813381732F622F94D0282FEA
:100CE000392FF12FE02F80819181F32FE22FE80F30
:100CF000F91F8B818083A981BA81E981FA8184817E
:100D000095810196FB2FEA2F848395838FEF90E0E6
:100D10008C839D8302C01C821D828C819D812596BF
:100D20000FB6F894DEBF0FBECDBFDF91CF911F91FC
:100D30000F910895CF93DF93CDB7DEB724970FB609
:100D4000F894DEBF0FBECDBF89839A831B821C82BD
:100D5000E981FA81A981BA8124813581FB2FEA2FAB
:100D6000828193812817390720F481E090E08B83FA
:100D70009C838B819C8124960FB6F894DEBF0FBEB6
:100D8000CDBFDF91CF910895CF93DF93CDB7DEB77D
:100D900022970FB6F894DEBF0FBECDBF89839A832A
:100DA000E981FA811482158222960FB6F894DEBF8B
:100DB0000FBECDBFDF91CF910895E62FF72FA82F5B
:100DC000B92F02C001900D9241505040D8F70895BC
:100DD000FF27EE27BB27AA2760FF04C0A20FB31F7F
:100DE000E41FF51F220F331F441F551F969587954B
:100DF0007795679589F70097760771F79F2F8E2F64
:100E00007B2F6A2F0895AA1BBB1B51E107C0AA1FA5
:100E1000BB1FA617B70710F0A61BB70B881F991F9B
:100E20005A95A9F780959095682F792F8A2F9B2F37
:100E30000895A1E21A2EAA1BBB1BEA2FFB2F0DC09F
:100E4000AA1FBB1FEE1FFF1FA217B307E407F5077A
:100E500020F0A21BB30BE40BF50B661F771F881F56
:100E6000991F1A9469F76095709580959095262F33
:100E7000372F482F592F6A2F7B2F8E2F9F2F0895A2
:00000001FF
